:030000000219FDE5
:03000B000200AA46
:03002B0002018748
:03005B0002033B62
:030073000203285D
:1000800002030406080C10182030406080040608A3
:100090000C10182030406080A0C00003070F1F0D17
:1000A0000D04050D050305030302C2AF306308C24A
:1000B0006385798AD2AF32C0D0C0E0206221E525C5
:1000C0006016E473E525F4C3334009758A00D263F2
:1000D000F57901D6F58AD262D0E0D0D0D2AF32C362
:1000E000E526334009758A00D263F57901F0F58A77
:1000F000C262E526F4602F30682520720DD0E0D072
:10010000D0C293C297C294D2AF32C293C297C29464
:10011000206F0C206509740CD5E0FDE57B4290D082
:10012000E0D0D0D2AF32758A00D263757900C28D2B
:10013000D262211F01C4306805206502D29301C438
:10014000306805206502D29401C43068052065023C
:10015000D29701C4C29230680A206507740CD5E0BA
:10016000FDD29301C4C29530680A206507740CD58E
:10017000E0FDD29401C4C29630680A206507740C71
:10018000D5E0FDD29701C4C2AFC2AD53E6EFC0D0F7
:10019000C0E0D2D3D2AFE57A6009E5776005757724
:1001A0000041D5757701C2CEE52A60072074491554
:1001B0002A21F87800790020742EE580307E01F441
:1001C00030E50278FF53DACF207E0343DA20307E19
:1001D0000343DA10C2D8C271E580307E01F430E505
:1001E0000279FFC3E89970CB306103752A18207437
:1001F00003752A18885CD27020740DE52B600415F5
:100200002B410843DA01C2D82070024177A85C2054
:100210006102C2702074367982B70431C3E894F069
:10022000400374F0F8E8C4540F28F87984B7030247
:10023000414DC313C3138721200802C313200A06AC
:10024000C3C898F8414D28F8500374FFF88822E598
:100250002D54066022206B1FE536C333C333F8E507
:1002600064C313C313F9C3952240028922E82522EF
:10027000F52250037522FF7882B60459852224A8FE
:1002800024C3E52495614002A861C3E89563400258
:10029000A8638825E566700241C8C3E8AA669A503B
:1002A00003E8FAE4F9EAC333FBE568F45B29400D9F
:1002B0002567F8E56760021567400B41C80AC3E58A
:1002C000679A5002056778FF8826C26FC3E52694B7
:1002D000F84002D26F20CF0AD0E0D0D043E610D24F
:1002E000AD32C2CF053AE57A6009E57860057578E8
:1002F00000611E7578017801E52A600530740215E9
:100300002AC3E55C94014005755F00611E756000BD
:10031000756900E55F2401F55F5003755FFFD0E06C
:10032000D0D043E610D2AD32C2AF53E67F7592FA19
:100330007593FFC260759104D2AF32C2AF53E6EF3E
:10034000C2ADC0D0C0E0C0F0D2D3D2AFA8FBA9FCF0
:10035000E57A6007C3E913F9E813F8C2D8307102EF
:1003600061AD53DACF207E0343DA10307E0343DAE7
:1003700020D271E580307E01F420E5026184882777
:100380008928A1DA53DACF207E0343DA20307E03B6
:1003900043DA10C2D8C271307402A1C67800E58079
:1003A000307E01F430E502A1C6885CA1AE53DACFFD
:1003B000207E0343DA20307E0343DA10C2712061CD
:1003C00002818653DACF207E0343DA10307E034366
:1003D000DA20C2D8D27188578958C3E89555F8E910
:1003E0009556F97B007E087A00C3E8948CE9940066
:1003F0005005755B008178882178A2E6A8216055B8
:10040000C3E894C8E994005008E4D2E4FB7A0A8176
:1004100053C3E89468E994015008E4D2E3FB7A0FEF
:100420008153C3E894D0E994025008E4D2E2FB7A05
:100430001E8153C3E894A0E994055008E4D2E1FB7F
:100440007A3C8153C3E89498E994085008E4D2E0D8
:10045000FB7A787E00C3E89559FCE9955AFD30E7B0
:100460000AECF42401FCEDF43400FD755B00C3ECF0
:0F0470009AED9E5003755B018859895A8557553F
:10047F008558567802A1AEC3E89527F8E99528F973
:10048F00307C02A192307B02A192307A02A18B20A4
:10049F00750281A9E9FDE8FC81C8E9C313F9E813E6
:1004AF00F8307902A18BE9C313F9E813F830780219
:1004BF00A18BE9C313FDE813FC20612CC3EC941C42
:1004CF00ED9402400281DFED701EC3EC94C850180A
:1004DF000529E52970021529C3E529940A5002A1BF
:1004EF00C6755C00D270A1C6E5296002152978880F
:1004FF00E6F97400207F087896B90302789EE62407
:10050F00FAFEE43400FFC3EC9EFCED9FFD9208B9A8
:10051F000310A2085007207609D276A13130760257
:10052F00C276A2085016B9030DECF42401FCEDF4C9
:10053F003400FD02054B78007900A192B90315EC48
:10054F0033FCED33FDC3EC940AFCED9400FD500435
:10055F007C007D00C3EC94FFED9400400678FF799A
:10056F0000A192EC8572F0A4C5F0A2F733F87900E0
:10057F0040030205AE78FF79000205AEE9C313F917
:10058F00E813F8307C0EE9600278FFC3E81338F8FF
:10059F00E43400F9C3E894FFE99400400278FF883F
:1005AF005CD270206102A1C6741FF4552F4BF52F3A
:1005BF00C274EB7002D274752A18307403752A0A4C
:1005CF00306102A1DA20740353DAFE207403752B15
:1005DF0006D0F0D0E0D0D0D2AD43E6103279010290
:1005EF00060A790302060A790A02060A791E02062A
:1005FF000A796402060A79C802060A7817E4D5E078
:10060F00FDD8FAD9F6227A147B780206317A107B5C
:10061F008C0206317A0D7BB40206317A0B7BC8024D
:10062F000631E573D5E001227902E4C295D5E0FDEC
:10063F00D294D5E0FDC294D5E0FDD295D5E0FDE989
:10064F0020E002D29330E002D297E573D5E0FDE9C6
:10065F0020E002C29330E002C2977496D5E0FDD934
:10066F00C9EAF8D5E0FDD8FBDBB8C29522C37C0000
:10067F007D0075F00005F0EA33FAEB33FB50F6EB33
:10068F0013FBEA13FAC3E9FFE8FEE89AF8E99BF9CE
:10069F005004EFF9EEF8B3EC33FCED33FDD5F0DF9A
:1006AF00EDF9ECF822E889F08A20D2D4F8A9F07B92
:1006BF000030F70B7BFFF42401F8E9F43400F9E87C
:1006CF008520F0A4ADF0F8E98520F0A4AFF0FEEDA1
:1006DF002EF974003FFA7C04C3EA13FAE913F9E820
:1006EF0013F8DCF48BF030F70AE8F42401F8E9F49E
:1006FF003400F9E889F0C2D4F8A9F0227882B60460
:10070F0003020766C3E55C940140030207308522AC
:10071F0024E4F544F545F546F547F548C26E020762
:10072F00667882E6FCD26EE522F523783879C7AA7F
:10073F0040AB41C3EB13FBEA13FAEC146013C3EBAA
:10074F0013FBEA13FAEC14146007C3EB13FBEA1361
:10075F00FAD17C8844894522C3E5449523F8E545C1
:10076F009400F9500CC3E89480E994FF40160207F7
:10077F0097C3E8947FE994005003020797787F7935
:10078F0000020797788079FF8849894A22E5492531
:10079F0046F8E54A3547F9854A20E4300701F43534
:1007AF0048FA30E709C3EA94F040150207D5C3EAC7
:1007BF00940F50030207D578FF79FF7A0F0207D500
:1007CF00780079007AF0C3E5249561500AC374016B
:1007DF009524500B0207F3E54A20E70E0207F3E5D5
:1007EF004A30E706884689478A482278A5E6FAC341
:1007FF00E54933F8E54A33F91206B4E930E70BC39C
:10080F00E89480E994FF4013012EC3E8947FE994A4
:10081F00005002012E787F7900012E788079FFE851
:10082F0020E715C3E52398F84009C3E89401400376
:10083F000208557801020855E8F424012523F840F1
:10084F000302085578FF884B2278A6E6FAA847A935
:10085F00481206B4E930E70CC3E89401E994FF406D
:0D086F001602088AC3E894FFE994005003C4
:10087C0002088A78FF790002088A780179FFE9205A
:10088C00E715C3E54B98F84009C3E894014003020F
:10089C0008B178010208B1E8F42401254BF84003B3
:1008AC000208B178FF88242278FF20692879A1E713
:1008BC006023E541601F74FF8541F0848539F03079
:1008CC006A0375F005A4F8C5F0600278FFC3E895DB
:1008DC00645002A864886322C3E54094C8E541943F
:1008EC0000E56350031401F5046002F5632202086D
:1008FC00FD2275E890227883E6FF30EDF9A8BDA9BA
:10090C00BE0570C3E57094084052757000E9FA7921
:10091C00A0E76044EA7007E571601B020936C3E882
:10092C0095716010E5715006600C14020942046068
:10093C00F9020942E571F571C39472401B7561C0EF
:10094C00C394044013756180C39404400B756140DB
:10095C00C39404400375610075BB0922E561241042
:10096C00500274FFF5617982B70402218FC3A8612C
:10097C00E524985002A824C3E895634002A8638834
:10098C00258826E570B4070375BB1022743279A74D
:10099C0087F0A4C5F0A2F733F8C3E895614002A82C
:1009AC0061882288248825882688642275400075F1
:1009BC0041F022C2AF75C820A8CCA9CDAA3A30CF3D
:1009CC00010A75C824D2AFC3EA13FAE913F9E81384
:1009DC00F8AB3BAC3C883B893CC3E89BF8E99C20DA
:1009EC00690A547FF930660241DC4136AD3D8A3DDF
:1009FC00F9EA9D547FFA600478FF79FFAE3EAF3F71
:100A0C008B3E8C3FA83BA93CC3E89EF8E99FF9C3F9
:100A1C00E54113FBE54013FAE82AF540E93BF541C3
:100A2C0050067540FF7541FF4183AA40AB41AC4075
:100A3C00AD417E047F02C3EB9404400D1E1FC3EB3B
:100A4C0094084005206A021E1FC3ED13FDEC13FC35
:100A5C00DEF7C3EA9CFAEB9DFBEF6009C3E913F9DF
:100A6C00E813F8DFF7EA28FAEB39FB8A408B4150A0
:100A7C00067BFF8B408B41C3EB94025002D2663055
:100A8C0069047F0341AE7892E6FFC3E53794824058
:100A9C00110FC3E53794A040010FC3EF9406400239
:100AAC007F057E02E541C4540FF9E541C454F0F8CA
:100ABC00E540C4540F28F8C3E89EFAE99400FB40C3
:100ACC0009C3EA9402EB940050047A02E4FB612817
:100ADC00AA40AB41EBC4FEEAC4540F4EFCC3EA9CE3
:100AEC00FAEB9400FBC3E813C313F8EA28FAEB34CF
:100AFC0000FB8A408B41C3EB94024002C266780231
:100B0C00EBC4FE7B00EAC4540F4EFAC3EA98FA40D9
:100B1C0005C3940250027A027892E6FF30600261BB
:100B2C0028855192855293D26043E680C3E49AF8AB
:100B3C00E49BF9C3E833F8E933F930660261BBE8AA
:100B4C00FAE9FBD3E913FDE813FC88518952C3EF92
:100B5C0094036038EF20E00DE82CF8E93DF9ECFA4D
:100B6C00EDFB020B84E828F8E939F9C3E82402F814
:100B7C00E93400F97AFE7BFFC3EF9403400E8A53ED
:100B8C008B54884D894E8C4F8D5061EF885389540E
:100B9C008A4D8B4E8C4F8D503069127553F07554B5
:100BAC00FF754FF07550FF7551F07552FF61EFE80E
:100BBC00FAD3E813FC8851C3EF94036020EF20E0D4
:100BCC0007E82CF8ECFA61DBE8282402F87AFEC37B
:100BDC00EF940340088A53884D8C4F61EF88538AF9
:100BEC004D8C4FE568C3335002646BF5683060027E
:100BFC0061F9753402D26043E680E52D5406602D10
:100C0C00A840A941C3E913F9E813F8306904E924B1
:100C1C0040F9C2AF53E67F759100C3E498F594E4B4
:100C2C0099F595759104D26043E680D2AF22D264D7
:100C3C00754300752000306C03752040020C59D2AE
:100C4C0064754300752040306C0375200078017981
:100C5C0001206620E52D54066002C2647914E5413A
:0D0C6C00C313700104F8C3941440027814FF
:100C7900306904781B791BC3E833F8C3E933F920D9
:100C89006010E543600C306903D53404D26DA110BE
:100C990091010543E59BF45440B5200281FA30697E
:100CA9000908C3E899400118818820640A08C3E843
:100CB90099400281598188C264C2AF53E67F759118
:100CC900003066127594007595F0759104D26043F1
:100CD900E680D2AF8159E5417EFFC3334009C33372
:100CE9004005C3334001FEC3E49E759400F5958128
:100CF900D3C3E5339401500281593064028159D834
:100D090002A10E8188C26DC2AF53E67F759100853D
:100D19005394855495759104854D92854E93D2606F
:100D290043E680D2AFE52D54066008206A020533F8
:100D3900020D4C306D0D206C0A2064071581158158
:100D49000216102278003064027801E53775F00741
:100D5900A4F9E5F028F5F0E9A2F013A2F113A2F243
:100D690013F537C394785003753778C3E537953849
:100D79004008D265C293C297C294306002A18385AC
:100D89004F92855093D26043E68022207D16C2AFF0
:100D9900754202C295D292306202D297D2AF759F44
:100DA90080020F83C2AF754202C295D296306202A9
:100DB900D293D2AF759F80020F83307243207D207A
:100DC900C2AF754203900165757B20C297C2963008
:100DD9006204D294A1E1D295D2AF759F89020F83A3
:100DE900C2AF754203900165757B20C293C29230F0
:100DF9006204D294C101D295D2AF759F81020F834B
:100E0900207D17C2AF754203900140C2973062023C
:100E1900D294D2AF759F89020F83C2AF75420390F6
:100E29000140C293306202D294D2AF759F81020F02
:100E390083207D16C2AF754204C292D296306202F7
:100E4900D294D2AF759F81020F83C2AF754204C29B
:100E590096D292306202D294D2AF759F89020F83E3
:100E6900307243207D20C2AF754205900154757BD5
:100E790004C294C295306204D293C187D292D2AF90
:100E8900759F80020F83C2AF754205900176757B0D
:100E990040C294C295306204D297C1A7D296D2AF0C
:100EA900759F80020F83207D17C2AF75420590019F
:100EB90036C294306202D293D2AF759F80020F83FB
:100EC900C2AF75420590014AC2943062EBD297D203
:100ED900AF759F80020F83207D16C2AF754206C28F
:100EE90096D295306202D293D2AF759F89020F8351
:100EF900C2AF754206C292D295306202D297D2AF82
:100F0900759F81020F83307243207D20C2AF7542E5
:100F190001900176757B40C293C292306204D297E8
:100F2900E12DD296D2AF759F81020F83C2AF754270
:100F390001900154757B04C297C296306204D29322
:100F4900E14DD292D2AF759F89020F83207D17C2DE
:100F5900AF75420190014AC293306202D297D2AF73
:100F6900759F81020F83C2AF754201900136C29706
:100F7900306202D293D2AF759F89C2652290013443
:100F8900757B00C293C297C294C292C296C295C29F
:100F99006222788076090876090876040876FF08BF
:100FA90076030876FF08760908760308760108763D
:100FB90001788C76010876FF0876FF0876FF0876B7
:100FC900FF0876FF0876030876FF0876FF0876FFA4
:100FD9000876250876D00876280876500876040819
:100FE90076FF08760208760008767A0876FF087692
:100FF90001087601087600087603087600227887CA
:10100900E6FFC272BF0302D2727888E6C394036016
:1010190008C27DE630E102D27DC27E7889E630E100
:1010290002D27EC3EF94026008758E01D27302105A
:101039003F758E00C273227880E614900080937801
:10104900A5F67881E6149000809378A6F67886E66E
:101059001490008D9378A7F67886E6F539C3940243
:0E1069005003753902789CE67538FFB4020317
:101077007538A0B4030375388278A3E61490009AF4
:1010870093F566120F8622227896E6FA7897E6FBA2
:101097007888E6B40305C3EB940EFB307F047A002F
:1010A7007BFFC3EB9AFCC3948250027C827572006B
:1010B7000572EC8572F0A4C3E5F0947D40F222D26C
:1010C7007F118F1205FB1205FB7A007B007C101243
:1010D70005F1E55C2AFA74003BFBDCF37C04C3EB07
:1010E70013FBEA13FADCF7FEC27F118F22757C002F
:1010F700757D00E5EF20E6037520000520903FFF92
:10110700E520146006901FFF1460009304600375C8
:10111700EF1653D9BF7581C043FF801205EC75EFF9
:101127000643B203E5B3240220E70DF521E5E320EA
:10113700E0068521B343E301120F867580FF75A48E
:101147000075F1F075D4DF75900275A5FC75F2FD99
:1011570075D50275A61075A0FF75F3F175E24112FA
:101167000F86E4F8F6D8FD756801120F9B12166911
:1011770078988673753001C2AF12060512061512EC
:1011870005FB12061C1205FB1206231205FBC2AF54
:10119700757C00757D0078FA79FA308507D9FBD818
:1011A700F7021C0011071140118E118F7898867372
:1011B700120F8675A90075B680757A007588107547
:1011C700890275C82475910475D84075A82275B829
:1011D7000275E690759B80759D0075D10E75BCC034
:1011E70075BB0975BA1175E8801205ECD2AF120804
:1011F700FA75360053DACF207E0343DA20307E03B8
:1012070043DA1043DA01C2D8C271120605D2617BF4
:10121700037A0CE55B70077A0CDB03021195120564
:10122700FB207003021195C270E55CC3940240E194
:10123700E52F541F855E5DF55EB55DD5DAD5C261D4
:1012470053DACF207E0343DA20307E0343DA10C21D
:10125700D8C27178A2E67008D274E52F54E0F52F52
:10126700C275752900120600307409C3E529940A6E
:101277004002D2751205F178023074027800C3E596
:101287005C9840F0C2AF120615120615120615D269
:10129700AF120605754C007888E6B4030261911217
:1012A70005F1788CE6C394015003021391E530C32E
:1012B70094015003021391757CA5757DF120743557
:1012C700C3E55C94FF5003021391C2AF12062AD202
:1012D700AF120600C3E55C940150EFC2AF120615CA
:1012E7001205F6120615D2AF120600C3E55C94FF8D
:1012F70040E90218157F02D27F118F120600C2AF94
:10130700C27F118FAE5CC3E55C947FD2AF500261A0
:10131700A11205ECC2AF12062AD2AFDFDA11C6C39B
:10132700EE7897F61206051217987F0AD27F118F6B
:10133700120600C2AFC27F118FAE5CC3E55C947F1B
:10134700D2AF50E61205ECC2AF1206151205F6121F
:101357000615D2AFDFD611C6EE24037896F6F879D4
:1013670097E7C394824003985006E824827897F65B
:101377001206051216AB1217C7120600118FC3E526
:101387005C94FF500241BE021815757C00757D0004
:10139700C3E55C954C4003855C4C120600780179E7
:1013A70088E7B403027805C3E55C984002419EC212
:1013B700AF12062A12062A12062AD2AF120605759E
:1013C7003000E4F531F5320531E531F4703F05328F
:1013D700789AE67819146012783214600D787D14C3
:1013E700600878FA146003753200C3E53298401D2F
:1013F700120F861205EC153275310078998673C283
:10140700AF12062AD2AF789886731206001205F635
:10141700E52A700530740221957801207402780658
:10142700C3E55C9840A17888E6C39403600312067D
:1014370000E52A7003021195C2AF120F86E4F52268
:10144700F523F524F525F526F567D2AF7885E6C3AC
:1014570033F565E4F544F545F546F547F548F57088
:0F146700F52CF52DF53775700875BB101205ECD7
:101476001208FE30EDFDA8BDA9BEE97001F888711D
:1014860012090275700875BB101107C2AF7561FFAE
:10149600120998852261852262852263D2AF752260
:1014A60001752401752501752601856069756A0136
:1014B60075B69075A903757A017888E6B40307C2F4
:1014C6007D307602D27DD268D269753300120EE085
:1014D600120F0F1209B81209BF1209B81209BF126A
:1014E60009B8120C4B12070B120D4D120D9412096E
:1014F600BF120C3A306E031207672066031208B457
:101506003066031208E4120D4D120DC31209BF1204
:101516000C4B306E0312079C120D4D120E3A120937
:10152600BF120C3A306E031207FA120D4D120E69F5
:101536001209BF120C4B306E03120858120D4D12D1
:101546000EE01209BF1208FE120C3A120D4D120FD0
:101556000F1209021209BF3069328564618564621F
:10156600856069756A0179187A0CC3E53399400F6D
:10157600C269D26A8A35856461856463021592C33D
:10158600E55C940140030214E8021618306A1D2037
:101596006C1AE535147006C26AD26B81E8F535C35C
:1015A600E55C940140030214E802161875360078CB
:1015B600FA79A4E760027803C3E55F985054307463
:1015C60004E52A604D7888E6B40317207D05207669
:1015D60007A1E8307602A1E8206C07D26C85646129
:1015E600A12778F0306C058564617820C3E54198C1
:1015F600500281E8306C1BC26CC27D307602D27D0F
:10160600D26A75351285646181E80536E55C60024B
:10161600C11B753600C2AF120F867887E6FE7602CA
:1016260011077887EEF6E4F522F523F524F525F57E
:1016360026F565752C00752D0075A90075B68075A3
:101646007A00D2AF120600120F8678A4E66006D2A0
:1016560092D295D296307409C3E53694044002219D
:101666009561C9901A0D78201216EDE520B4550C37
:10167600A31216EDE520B4AA0302168B120F9B12D5
:1016860016AB0216AA901A0378807B0A1216EDA3EF
:1016960008DBF9901A0F788C7B191216EDA308DB7C
:1016A600F9901A2822C2AF12173012170D901A009D
:1016B600740E1216F2A374071216F2A374151216FC
:1016C600F2901A0378807B0A1216F1A308DBF990D0
:1016D6001A0F788C7B191216F1A308DBF91217433F
:1016E600121721901A2822E493F622E6438F01531B
:1016F6008FFDFFC3E583941C400122EF857CB785EF
:101706007DB7F0538FFE22438F02438F01857CB74E
:10171600857DB7901A0DF0538FFC22901A0D7455E3
:10172600D1F2901A0E74AAD1F2227A3079D07820AA
:10173600901A40D1EDE520F709A3DAF7227A30793D
:10174600D0901A40E7D1F209A3DAF922AB74A87552
:10175600BB01027980BB02027981BB03027982BB9D
:1017660004027984BB05027986BB06027992BB071F
:10177600027987BB080279A3BB0902799CBB0A02DE
:101786007988BB0B027989E8F7227C05120605DC0D
:10179600FB22C2AF12061512061C12062312062AD7
:1017A6001205F612061512061C12062312062A1236
:1017B60005F612061512061C12062312062AD2AFC9
:1017C60022C2AF12062A12062312061C1206151290
:1017D60005F612062A12062312061C120615120513
:1017E600F612062A12062312061C120615D2AF227C
:1017F600AE74AF75C2AF1206151206151206151293
:1018060005F6DEF212062A1205F6DFF8D2AF22122C
:1018160017981217901217907574017575017576E1
:10182600001217F67C05AD5C120605C3ED955C70DB
:10183600F5C3E55C9401400AC3E55C94FF403702BA
:1018460018591217521216AB121798C2AF75EF1627
:10185600121790DCD10576C3E5769403500280C159
:0F1866001217900575E5741490009F93F808C34E
:10187500E57598500280A81217901217900574C349
:10188500E574940C50028094120F9B1216ABC2AFF4
:0618950075EF161217901A
:0319FD000210F4E1
:101A00000E0715090904FF03FF0903010155AA0187
:101A1000FFFFFFFFFF03FFFFFF25D0285004FF0259
:091A2000007AFF0101000300FF40
:101A40002358526F746F723430412320202020209D
:101A500023424C48454C492346333930232020202B
:101A60002020202020202020202020202020202076
:101C0000C2AFC2D353D9BF7581C043B20343FF8073
:101C1000752438752503B1DC7529A5752AF175E29F
:101C20004043F12053A4DF75D4FFD2857DFA7803B9
:101C300079E67C10752200752300901DE97B0675FE
:101C400024987525013085028145208508D8FBD967
:101C5000F9DCF781B7308508D8FBD9F9DCF781B713
:101C6000B19CE493A3C39A6004DDC381B7DBDBB10D
:101C70008E6002812E7B08E493FAA3B16FDBF87AC1
:101C800030B16F752200752300B18EEAFCEBFDC305
:101C9000ED94FE400EB18E8A278B28ED30E0048A49
:101CA000828B83B18E7AC270D8C3ED94FE601950D6
:101CB000CEBD002BEC600F7520007521FF7529004B
:101CC000752A000200008100A827A9280809D80465
:101CD000D90281DCB192EA89AAF281CE0D81A3C337
:101CE000ED94035053EDA2E092007AC5C3E58294CF
:101CF00000E583941C508A200010438F02438F011B
:101D00008529B7852AB7F0300029A827A92808090E
:101D1000438F01538FFDD804D902A133C3E58394C7
:101D20001C4003A3A11689AAE28529B7852AB7F02A
:101D3000A3A116538FFC817F7AC1BD030CE493A34A
:101D4000FAB153DCF8B14B817F8181AA22AB23B178
:101D50006FEBFAEA6222752608C3E52313F523E543
:101D60002213F52250066323A0632201D526EAB18F
:101D7000DCB1DC75260AEAF4200102D285300102CA
:101D8000C285B1DCC3134002C201D526EB22B19259
:101D9000EAFB208502A192308502A197752608AE44
:101DA00024AF25C3EF13FFEE13FEB1E0B1DCC3EAAD
:101DB000133085024480FA30E703632201C3E52330
:101DC00013F523E52213F52250066323A0632201B5
:101DD000D526D9E52265236523F52222AE24AF2539
:101DE0000E0FDEFEDFFCD20122424C48656C6934E6
:071DF000373163F390060197
:00000001FF
